:020000000829CD
:02000800E828E6
:04000C000D08820752
:10001000003407340F340034FF340D0882070034F5
:1000200007340F340234FF340D08820700340734DC
:100030000F340434FF340D088207003407340F34C2
:100040000834FF340D088207003407340F341034AD
:10005000FF340D088207003407340F342034FF3496
:100060000D088207003407340F340534FF340D08BF
:100070008207003407340F340934FF340D08890037
:10008000831608148312080808000D088207093433
:1000900002340034FF340D088207183402340A3465
:1000A0003E340A343E3431340034FF34913095000C
:1000B0000A307E2009307E2000308D0085195E28B0
:1000C0000D088900060888008E0083160815553033
:1000D0008900AA308900881408118312851D6E28B2
:1000E0000608FF3A03197728AA208D0A5E280330F4
:1000F0008E009000FF309500AA207D288C008D0195
:1001000003100C0D8207062098280D209828142033
:1001100098281B20982822209828292098283020C9
:100120009828372098283E209828452098284B204A
:100130008E008E080319A628FF300E06031908004A
:10014000AA208D0A02308F00D520802804308F002D
:10015000D520A12803108E0C8E0803190800031C5B
:10016000BA280330900001308F008514C22085101A
:10017000D520AA28013090008F008514C220851058
:10018000D520AA2810089100150892000514B23055
:100190009300930BC9280510B2309300930BCE281F
:1001A000920BC628910BC42808000F08910015086F
:1001B00092001414B2309300930BDC281410B23068
:1001C0009300930BE128920BD928910BD7280800B4
:1001D0009600030E9700980B022910309800990B97
:1001E00002293C309900A40BFA280A30A4009E038F
:1001F000031920149C0AA0141C081D02031D0229C7
:1002000001309C000B11170E8300960E160E09008C
:10021000073062008501860118306500FF306600F6
:100220008519562801308A001529810164008B0147
:100230008B178B16103098003C3099000A30A400C0
:10024000A0012B219E08031D732160309E007E219A
:100250008B13630000000608073930219E003929FE
:10026000820700340334063409340C340F3412345A
:100270001534060838399A0003109A0C9A0C9A0C17
:100280001A0847219F001A085021A1005929820706
:1002900000340134023403340434053406340734A2
:1002A0008207013401340234033404340534063443
:1002B00007349A01061F5D291A14861F60299A14B3
:1002C000051E63291A151A085021013E9D001D08BC
:1002D000210203186C21080018080239031D851437
:1002E000031985106C29201018080F39031985147B
:1002F000031D8510201C74298510080001309C0006
:10030000A00120111C082106031D20152019812998
:10031000A01005159130950000308A001F087E203E
:100320001908363A031D90291F087E201908303A13
:10033000031D96291F087E2019082A3A031D9C29AF
:100340001F087E201908243A031DA2291F087E20B9
:1003500019081E3A031DA8291F087E201908183AFB
:10036000031DAE291F087E201908123A031DB42967
:100370001F087E2019080C3A031DBA291F087E2089
:100380001908063A031DC0293C30950009307E202B
:1003900008307E2001308A00A01CCC29051181295B
:02400E00F13F80
:0E42000014000F00190011000F001900FF003C
:00000001FF
